:100000000C94AC040C94F4040C94F4040C94F404D8
:100010000C94F4040C94F4040C94F4040C94F40480
:100020000C94F4040C94F4040C94F4040C94B01B9D
:100030000C94F4040C94871B0C94F4040C94811F0E
:100040000C94F4040C94F4040C94F4040C94611BCC
:100050000C94F4040C94F4040C94F4040C945F1FBA
:100060000C94F4040C94F4040C94F4040C94F40430
:100070000C94F4040631FF0974A1010975150026DA
:10008000FF009520750881020976150026FF00956E
:100090002075089102C005010902A1010901A10012
:1000A0008501050919012908150025019508750123
:1000B00081020501093009311581257F95027508F6
:1000C000810609381581257F950175088106050C83
:1000D0000A38021581257F950175088106C0C00583
:1000E000010980A10185021601002637001A81004E
:1000F0002AB700751095018100C0050C0901A10106
:100100008503160100269C021A01002A9C02751024
:1001100095018100C005010906A101050719E02923
:10012000E715002501950875018102950175088183
:1001300001050819012905950575019102950175BB
:100140000391010507190029FF150026FF009506F8
:1001500075088100C00A00722530325820007325CE
:10016000303258200025303258200025583A2530AA
:10017000386225730A000A20203031323334353694
:10018000370A004C45443A20253032580A000A4CC0
:100190006F6F702073746172742E0A000A55534297
:1001A00020636F6E666967757265642E0A000A5473
:1001B0004D4B3A6266383266312F4C5546413A64AF
:1001C00036613764660A0009025400030100A03258
:1001D00009040000010301010009211101000122AD
:1001E00040000705810308000A090401000103011A
:1001F0000200092111010001227F00070582030886
:10020000000109040200010300000009211101009E
:1002100001222200070583032000011201100100C2
:10022000000008EDFE21500101010200013A0353D4
:10023000004F004E00590020004E0045005700536B
:100240000020006B006500790062006F00610072A1
:10025000006400200063006F006E0076006500728D
:10026000007400650072000000080354004D004B4C
:100270000000000403090473797374656D3A202546
:100280003034580A00636F6E73756D65723A2025BD
:100290003034580A003F004D3E2000433E20000A03
:1002A00000257500363A20776865656C5F74696D66
:1002B000655F746F5F6D61783A20000A00257500F4
:1002C000353A20776865656C5F6D61785F7370653E
:1002D00065643A20000A00257500343A2074696D7F
:1002E000655F746F5F6D61783A20000A00257500C4
:1002F000333A206D61785F73706565643A20000A57
:1003000000257500323A20696E74657276616C283A
:100310006D73293A20000A00257500313A20646582
:100320006C6179282A31306D73293A20000A092D31
:100330002056616C756573202D0A004D3E004D25D9
:10034000643E20003F007365742064656661756CCF
:10035000740A00433E20000A002530325820006B0A
:100360006579626F6172643A2000803A3B3C3D3EA1
:100370003F40414243291E1F2021222324252627B6
:100380002D2E742A2B141A0815171C180C12132F53
:10039000304C78041607090A0B0D0E0F333432283F
:1003A000791D1B0619051110363738757D7A397796
:1003B0002C7665007C5F6061565C5D5E57595A5BC8
:1003C000666252635850514F8080808080805554BF
:1003D000678044454A494D4B4E80808080808080B4
:1003E00080808080038080808080290A00257500BD
:1003F0002F002575005D280025640020002564007D
:10040000200025640020002564007C00253032583F
:10041000006D6F7573656B6579205B62746E7C78B7
:100420002079207620685D287265702F61636C29C1
:100430003A205B006D6F7573653A205B253032584A
:100440007C25642025642025642025645D0A000A3B
:10045000092D204D61676963202D0A643A0964659E
:100460006275670A783A096465627567206D617420
:100470007269780A6B3A096465627567206B657901
:10048000626F6172640A6D3A096465627567206D16
:100490006F7573650A763A0976657273696F6E0ACD
:1004A000733A097374617475730A633A09636F6E02
:1004B000736F6C65206D6F64650A302D343A096C7A
:1004C00061796572302D34284631302D4634290A41
:1004D000506175733A09626F6F746C6F6164657215
:1004E0000A000A092D20436F6E736F6C65202D0A78
:1004F0004553432F713A09717569740A6D3A096D54
:100500006F7573656B65790A003F0074696D65727C
:100510005F72656164333228293A202530346C5883
:100520000A006B6579626F6172645F69646C653A39
:100530002025580A006B6579626F6172645F707282
:100540006F746F636F6C3A2025580A00686F73747C
:100550005F6B6579626F6172645F6C656473282993
:100560003A2025580A000A092D20537461747573C6
:10057000202D0A004743433A20372E332E302041A6
:1005800056522D4C4942433A20322E302E302041D3
:1005900056525F415243483A2061767233350A0021
:1005A0004F5054494F4E533A204C554641204D4FE1
:1005B0005553454B45592045585452414B455920B8
:1005C000434F4E534F4C4520434F4D4D414E4420D9
:1005D0004B45594D41505F53454354494F4E20348C
:1005E0003039360A004255494C443A206266383266
:1005F0006631202831313A35353A3435204E6F7620
:100600002020392032303233290A005649443A201A
:1006100030784645454428544D4B29205049443AAA
:100620002030783530323128534F4E59204E4557BF
:1006300053206B6579626F61726420636F6E7665BB
:100640007274657229205645523A20307830313024
:10065000310A00444553433A20636F6E76657274E5
:100660007320534F4E59204E4557532070726F746C
:100670006F636F6C20696E746F205553420A000AD5
:10068000092D2056657273696F6E202D0A000A6D60
:100690006F7573653A206F66660A000A6D6F757331
:1006A000653A206F6E0A000A6B6579626F61726449
:1006B0003A206F66660A000A6B6579626F61726440
:1006C0003A206F6E0A000A6D61747269783A206F81
:1006D00066660A000A6D61747269783A206F6E0A64
:1006E000000A64656275673A206F6E0A000A6465E5
:1006F0006275673A206F66660A000A0A626F6F7455
:100700006C6F616465722E2E2E2000433E20006DBA
:100710006B5F776865656C5F74696D655F746F5F4B
:100720006D6178203D2025640A006D6B5F776865F8
:10073000656C5F6D61785F7370656564203D202531
:10074000640A006D6B5F74696D655F746F5F6D61E6
:1007500078203D2025640A006D6B5F6D61785F73C2
:1007600070656564203D2025640A006D6B5F696ECD
:1007700074657276616C203D2025640A006D6B5FA4
:1007800064656C6179203D2025640A006D6B5F779C
:100790006865656C5F74696D655F746F5F6D6178C6
:1007A000203D2025640A006D6B5F776865656C5F8E
:1007B0006D61785F7370656564203D2025640A0073
:1007C0006D6B5F74696D655F746F5F6D6178203DFF
:1007D0002025640A006D6B5F6D61785F73706565DD
:1007E00064203D2025640A006D6B5F696E7465723C
:1007F00076616C203D2025640A006D6B5F64656C3A
:100800006179203D2025640A00776865726520645F
:10081000656C74613A20637572736F723D25642C48
:1008200020776865656C3D25640A536565206874AA
:1008300074703A2F2F656E2E77696B6970656469E5
:10084000612E6F72672F77696B692F4D6F757365B6
:100850005F6B6579730A000A092D204D6F7573650A
:100860006B6579202D0A4553432F713A09717569DB
:10087000740A313A0964656C6179282A31306D73E4
:10088000290A323A09696E74657276616C286D7353
:10089000290A333A096D61785F73706565640A34BB
:1008A0003A0974696D655F746F5F6D61780A353AF6
:1008B00009776865656C5F6D61785F737065656405
:1008C0000A363A09776865656C5F74696D655F74AF
:1008D0006F5F6D61780A0A703A097072696E7420F0
:1008E00076616C7565730A643A0973657420646592
:1008F0006661756C74730A75703A092B310A646FFE
:10090000776E3A092D310A706775703A092B3130CC
:100910000A7067646F776E3A092D31300A0A737076
:10092000656564203D2064656C7461202A206D61DA
:10093000785F7370656564202A2028726570656130
:1009400074202F2074696D655F746F5F6D61782905
:100950000A004C25640A000011241FBECFEFD4E02A
:10096000DEBFCDBF04B603FE28C08091DA039091AC
:10097000DB03A091DC03B091DD038730904BA740EF
:10098000B04BD9F41092DA031092DB031092DC031F
:100990001092DD0314BE0FB6F894A8958091600004
:1009A000886180936000109260000FBE1092010871
:1009B00010920008E0E0F8E3099511E0A0E0B1E052
:1009C000EEE9F2E402C005900D92A233B107D9F727
:1009D00023E0A2E3B1E001C01D92AA3DB207E1F716
:1009E0000E947F1C0C944D210C940000FF93EF9308
:1009F000E0913201F0913301309709F00995EF91C0
:100A0000FF910895FC018591803011F0EFDFFBCF5D
:100A10000895FF27E0E230E247FF0CC0419597FFC1
:100A200009C0EDE26095709580959095611D711DEE
:100A3000811D911D27FF02C0219530E350E2AA27B6
:100A4000660F771F881F991FAA1FA41710F0A41BF9
:100A500063955A95A9F7AA3008F0A95FA05DAF93F6
:100A6000F395611571058105910541F7ED3211F49A
:100A7000EF93F395F21718F43F93F395FBCF8F9113
:100A8000B5DFFA95E1F70895E991F9918591803004
:100A900021F0853219F0AADFF9CF089520E0E8941B
:100AA00055915532C1F3503311F4689455915A332E
:100AB00048F4505390F3220F022E220F220F200DE4
:100AC000250FF4CF0EF4219589919991533619F39E
:100AD000533729F1533559F1BC0188279927E894F8
:100AE0005C3621F48991999168945591543639F482
:100AF00046EF7EF077FF0DC08FEF9FEF0AC05537AE
:100B00004AE039F0583540E121F0523642E009F030
:100B10000895FF93EF937DDFEF91FF91B7CFFF93A0
:100B2000EF93FC0181918030B9F360DFFBCFFF933D
:100B3000EF9368DFF1CFDF93CF93CDB7DEB7259684
:100B4000A3DFCF91DF910895803FC1F48091CC0362
:100B500087FD1092CC038091CB0381110EC0809150
:100B6000CC0381110AC08091CD03811106C0809110
:100B7000CE03811102C01092C5030895813F29F46C
:100B80008091CC0318162CF3E6CF9091CB03823FD3
:100B900029F497FFE0CF1092CB03DDCF833F19F408
:100BA0001916CCF3D8CF893F39F48091CD031816AC
:100BB00094F61092CD03CFCF8A3F29F48091CD03D4
:100BC00087FFC9CFF6CF8B3F39F48091CE0387FFE3
:100BD000C2CF1092CE03BFCF8C3F29F48091CE03B9
:100BE0001816BCF3B8CF843F31F48091CA038E7FCE
:100BF0008093CA03B0CF853F21F48091CA038D7FD3
:100C0000F7CF863F21F48091CA038B7FF1CF873FD6
:100C100021F48091CA03877FEBCF883F21F4809134
:100C2000CA038F7EE5CF8D3F31F48091C4038E7F60
:100C30008093C40390CF8E3F21F48091C4038D7FB5
:100C4000F7CF8F3F09F087CF8091C4038B7FF0CF20
:100C50008091C40380FF0CC06091130170E0759512
:100C60006795759567956115710559F1862F0895FA
:100C700081FF06C06091130170E075956795F3CF11
:100C80006091130170E082FD0CC06091C503662382
:100C9000A9F0209112018091130190E0621730F0C9
:100CA000BC0160387105F8F28FE7089570E00E948A
:100CB0000E21622F70E00E941F21F3CF61E070E0EF
:100CC000D5CF81E008958091C40380FF11C0809149
:100CD000150190E065E070E00E940E2195958795E2
:100CE0009595879580389105B0F50097B1F10895F5
:100CF00081FF0AC08091150190E065E070E00E94DC
:100D00000E2195958795EECF82FF08C08091150141
:100D100090E065E070E00E940E21E4CF3091C503C1
:100D20003323B1F0209114018091150190E065E02A
:100D300070E00E940E21BC013217A0F6832F90E0D4
:100D40000E940E21622F70E00E941F21CB01CACFAA
:100D500085E090E008958FE7089581E00895803F51
:100D600031F40E94630681958093CC030895813FFE
:100D700019F40E946306F8CF823F31F40E946306A3
:100D800081958093CB030895833F19F40E946306F5
:100D9000F8CF893F29F40E9428068093CD03089557
:100DA0008A3F21F40E9428068195F7CF8B3F31F4CA
:100DB0000E94280681958093CE0308958C3F19F4F4
:100DC0000E942806F8CF843F31F48091CA038160E5
:100DD0008093CA030895853F21F48091CA038260FD
:100DE000F7CF863F21F48091CA038460F1CF873F1B
:100DF00021F48091CA038860EBCF883F21F4809171
:100E0000CA038061E5CF8D3F31F48091C4038160D6
:100E10008093C40308958E3F21F48091C4038260BF
:100E2000F7CF8F3FB9F78091C4038460F1CFE72FEC
:100E3000F0E093E0EE0FFF1F9A95E1F7E60FF11D4A
:100E4000E659FC4F6491E62FE295E77090E023E0CD
:100E5000880F991F2A95E1F78E0F911D34E0880FB6
:100E6000991F3A95E1F7E62FEF70E80FF92FF11D82
:100E7000EE0FFF1FE050F8498591949108952FB728
:100E8000F8948091CF039091D003A091D103B091B9
:100E9000D2032FBF08954F925F926F927F929F92DD
:100EA000AF92BF92CF92DF92EF92FF920F931F9378
:100EB000CF93DF9300D000D01F92CDB7DEB76B8306
:100EC0007C838D837A018C819D81892B49F08FEF02
:100ED000F81204C081E09FEF491719F080E001C0CB
:100EE00081E080FD6AC00F2D10E0CE2CD12C8B81CB
:100EF000882309F456C040903C0350903D03609015
:100F00003E0370903F038091D6039091D703A09148
:100F1000D803B091D903482A592A6A2A7B2A2FE19B
:100F2000A22EB12C9A2CD301C2010A2C04C0B69572
:100F3000A795979587950A94D2F780FD2BC081E0FD
:100F4000A81AB10878F7912CF80193E0EE0FFF1F73
:100F50009A95E1F7E05CFC4FEC0DFD1D9082E98273
:100F6000FA8269817A81892D0F900F900F900F90EE
:100F70000F90DF91CF911F910F91FF90EF90DF9035
:100F8000CF90BF90AF909F907F906F905F904F9069
:100F90000C941707B7018A2D0E941707019779F261
:100FA000D3CFF80183E0EE0FFF1F8A95E1F7E05CF5
:100FB000FC4FEC0DFD1D9080D2CF90E080E00F90B3
:100FC0000F900F900F900F90DF91CF911F910F9185
:100FD000FF90EF90DF90CF90BF90AF909F907F9069
:100FE0006F905F904F90089541E050E060E070E0B6
:100FF00004C0440F551F661F771F8A95D2F740958E
:1010000050956095709580913C0390913D03A0911F
:101010003E03B0913F0384239523A623B7238093F7
:101020003C0390933D03A0933E03B0933F03089588
:1010300041E050E060E070E004C0440F551F661FBF
:10104000771F8A95D2F780913C0390913D03A09140
:101050003E03B0913F03842B952BA62BB72B809397
:101060003C0390933D03A0933E03B0933F03089548
:1010700080913B0390910A03981301C008958F5FFC
:101080008770FACF1F93CF93DF9300D000D01F92C9
:10109000CDB7DEB7942F4983252F5A836B837C838A
:1010A0008D834C815D8181E0452B31F02F3F19F418
:1010B00081E09F3F09F080E0182F117080FD2CC067
:1010C00049815A816B817C818D810E944B07292F38
:1010D00022952F702C3078F42A30A8F42250223038
:1010E000C8F0812F0F900F900F900F900F90DF910D
:1010F000CF911F9108952C3011F02F3091F793FB71
:10110000112710F9EECF803C28F0803E50F3815F2C
:10111000833038F311E0E5CF10E0E3CFE091C60370
:10112000F091C703309721F00190F081E02D0994F0
:1011300080E008951092E2001092E100E0EEF0E00D
:10114000808181608083E8EDF0E080818F7780830B
:1011500019BCE3E6F0E08081816080831092E802B0
:1011600008950E949A08F89487E797E790930108FA
:101170008093000887E090EBDC018093DA03909382
:10118000DB03A093DC03B093DD0388E19CE00FB6A2
:10119000F894A895809360000FBE90936000FFCFF5
:1011A000FC018091FC029091FD0286179707A0F048
:1011B0006115710529F49091E8009E779093E800FD
:1011C00090E06115710551F4911108C08091E8001B
:1011D00082FF32C080E00895BC01F2CF8091FE0210
:1011E0008823B1F18530B1F18091E80083FD2EC0F4
:1011F0008091E80082FDEACF8091E80080FFE1CF96
:101200002091F20030E06115710519F028303105A8
:1012100058F091E02830310509F090E02091E80085
:101220002E772093E800CDCF81918093F10061501B
:1012300071092F5F3F4FE7CF8091FE02882341F075
:10124000853041F08091E80083FFC0CF81E00895B0
:1012500082E0089583E008952091E4003091E50054
:1012600085E69091EC0090FF06C09091E80090FF19
:1012700006C080E008959091E80092FDFACF909129
:10128000FE02992391F0953091F09091EB0095FD3D
:1012900010C04091E4005091E5002417350709F390
:1012A00081509A01F1F684E0089582E0089583E088
:1012B000089581E008958091F60287FF13C0809120
:1012C000E80082FF06C08091E8008B778093E800F9
:1012D00004C08091FE028111F2CF08958091FE0238
:1012E0008823D9F38091E80080FFF8CF8091E8004F
:1012F0008E77ECCF982F9093E900242F762F50E033
:10130000891731F07091EC002091ED005091F000C0
:1013100021FD07C09F5F953071F78093E90081E060
:1013200008953091EB003E7F3093EB003091ED005B
:101330003D7F3093ED003091EB0031603093EB0056
:101340007093EC002093ED005093F0002091EE009C
:1013500027FDE0CF80E008950F931F93CF93DF9395
:10136000CDB7DEB7AA970FB6F894DEBF0FBECDBFDC
:101370008091FE02882309F44EC11091E9001F708C
:101380008091EC0080FF39C080E8182B1092E900B2
:101390008091E80083FF3CC1E6EFF2E08EEF92E03F
:1013A0002091F10021938E179F07D1F78091F702CA
:1013B000833009F470C018F5813009F447C08230D9
:1013C00009F4DAC08091E80083FF14C18091F6022D
:1013D0009091F7029A3008F00DC1E92FF0E0ED503E
:1013E000F64F0C943321CD0AF30AFA0AF30AFA0AEB
:1013F000550B770BFA0A720C7F0C80E0C6CF8A304F
:1014000009F4A9C08B3009F47DC08930D9F68091E8
:10141000F6028132B9F68091FA029091FB02892B93
:1014200089F68091E800877F8093E8008091E8004A
:1014300082FF2CC08091F1008093EA028091E80045
:101440008B778093E8000E945B09BCCF8091F60205
:10145000813A09F0B7CF8091E800877F8093E80058
:101460008091FA029091FB02892B61F060E090E09C
:1014700080E070E00E94D0088091E8008B77809334
:10148000E800A0CF68E08BEE92E0F3CF8091FE02FF
:101490008111CCCF97CF8091F602813A09F092CF9B
:1014A0008091FA029091FB02892BA1F48091E800CF
:1014B000877F8093E8008091E80080FFFCCF8091D7
:1014C00011018093F1008091E8008E778093E8000D
:1014D0000E945B098091FA029091FB02019709F04A
:1014E00071CF8091E800877F8093E8008091E800C9
:1014F00080FFFCCF809110018093F1008091E80083
:101500008E779FCF8091F602813209F05BCF809178
:10151000FA029091FB02892B59F48091E800877FB1
:101520008093E8000E945B098091F802809311018A
:101530008091FA029091FB02019709F043CF8091CC
:10154000E800877F8093E8000E945B098091F802A1
:101550008093100137CF8091F602813209F032CFAB
:101560008091E800877F8093E8000E945B0980916A
:10157000F9028093D30326CF8091F602813A09F0D5
:1015800021CF8091E800877F8093E8008091E80078
:1015900080FFFCCF8091D303AFCF803889F08238B1
:1015A00049F58091FA028F70853020F58093E9002B
:1015B0008091EB0085FB882780F91092E90006C036
:1015C0008091F3029091F402911182609091E80071
:1015D000977F9093E8008093F1001092F100809142
:1015E000E8008E7731C0282F2D7F21F48823F1F079
:1015F000823079F18091E80083FF0AC08091E80091
:10160000877F8093E8008091EB0080628093EB00FD
:101610001F701093E900AA960FB6F894DEBF0FBEB4
:10162000CDBFDF91CF911F910F9108958091F80266
:10163000813001F7933009F080E08093F40210923A
:10164000E9008091E800877F8093E8000E945B09B1
:10165000D1CF8091F8028111F2CF8091FA028F7080
:101660002FEF280F243030F68093E9002091EB0013
:1016700020FFE5CF933031F48091EB0080628093BE
:10168000EB00DDCF9091EB0090619093EB0021E0B7
:1016900030E001C0220F8A95EAF72093EA00109209
:1016A000EA008091EB008860EACF8111A3CF00911E
:1016B000F8020F778091E3008078802B8093E3001D
:1016C0008091E800877F8093E8000E945B09809109
:1016D000E80080FFFCCF8091E30080688093E30006
:1016E00083E0011101C082E08093FE0283CF805825
:1016F000823008F07FCF2091F8023091F9022C3D22
:1017000083E03807A1F583E08A838AE289834FB7B3
:10171000F894DE01139620E03EE051E2E32FF0E082
:1017200050935700E49120FF03C0E295EF703F5FB4
:10173000EF708E2F90E0EA30C0F0C7968D939D93A6
:101740002F5F243159F74FBF8091E800877F809346
:10175000E8006AE270E0CE0101960E94D008809114
:10176000E8008B778093E80045CFC096E7CF809163
:10177000FA029091FB02432F55274330510509F49B
:101780004FC078F54130510509F445C084E590E03B
:10179000E7ECF1E04230510509F02CCF2091E80050
:1017A000277F2093E8002091FC023091FD028217F0
:1017B000930708F49C0140E02115310509F063C04E
:1017C000411161C08091E80082FDC9CF8091FE0285
:1017D000882329F2853019F28091E80083FFF2CF47
:1017E000BECF4132510509F43FC04232510509F0E4
:1017F00001CF8330910508F0FDCEFC01EE0FFF1FF5
:10180000E45EFE4F0190F081E02D875E9E4FDC018B
:101810008C9190E01DC082E190E0EBE1F2E0BECF60
:10182000332721303105C1F060F02230310509F055
:10183000E1CEEDE2F2E0E4918E2F90E0EDE2F2E015
:1018400007C0E3E7F2E0E4918E2F90E0E3E7F2E0F7
:10185000009709F4CFCEA2CFE9E6F2E0E4918E2F13
:1018600090E0E9E6F2E0F4CF8330910508F0C2CED3
:10187000880F991FFC01EE5DFE4F0190F081E02D75
:1018800089E090E08BCF8091FE02882309F467CF36
:10189000853009F464CF8091E80083FD60CF8091AA
:1018A000E80082FD8FCF8091E80080FF85CF809196
:1018B000F20090E02115310519F08830910550F0C3
:1018C00041E0089709F040E08091E8008E7780932E
:1018D000E80072CF44914093F100319621503109D4
:1018E0000196E8CF803809F085CE8091E800877FA7
:1018F0008093E8008091F5028093F10070CE811111
:1019000079CE0091F802023008F074CE8091E800A0
:10191000877F8093E8000093F5020E945B09002313
:1019200099F084E08093FE0242E061EC81E00E9445
:101930007A0942E061EC82E00E947A0946E261ECB9
:1019400083E00E947A0956CE8091E30087FDE9CFBB
:1019500081E0E8CFEF92FF920F931F93CF937C012A
:101960008B010E942C09C82F811119C08091E800B9
:1019700085FD0DC08091E8008E778093E8000E947D
:10198000AC090E942C09882389F3C82F08C0F701ED
:1019900081917F018093F1000150110939F78C2F5B
:1019A000CF911F910F91FF90EF9008958091EA02DF
:1019B00008958091C302811113C09FB7F89440919C
:1019C000CF035091D0036091D1037091D2039FBF98
:1019D000443C59406105710518F081E08093C302D1
:1019E0000895EF92FF920F931F93CF93DF93D82F19
:1019F0000FB607FE46C08091FE02843079F08091D8
:101A0000030190E001962091050130E082239323A9
:101A1000209104012817190609F0C9C00E94D90CA9
:101A200081110FC08091030190E001962091050182
:101A300030E082239323209104012817190609F02E
:101A4000B6C00E943F078C01C091E900CF70809121
:101A5000EC0080FD37C080E0C82B83E08093E90074
:101A600085E0E82E8091EB0085FD08C08091EB00B9
:101A700080FF04C08091EE0087FD44C0CF70C0930A
:101A8000E900E09103018E2F90E00196209105017D
:101A900030E082239323209104012817190609F4CA
:101AA0007EC08091010190910201E80FF92FF11D94
:101AB000D083809103018F5F9091050189238093EA
:101AC00003016DC080E8C8CFE0910101F0910201EF
:101AD000E80FF11D90818F5F209105018223809393
:101AE00004019093F1008091E80085FD0BC0809186
:101AF000E80080FF07C08091E8008E778093E800BF
:101B0000E09200018091040190910301981741F146
:101B10009091E80095FDD8CF80E029C01092F100A7
:101B20002EC08091030190E001962091050130E0E4
:101B300082239323209104012817190609F09ECFD0
:101B4000F0900001FF2009F499CF0E943F07801711
:101B5000910709F487CFFA94F09200018C0182CFAB
:101B60008091E80085FFD8CFD093F10081E090917B
:101B7000F200992379F09091E80090FF0BC09091CA
:101B8000E80095FDCBCF9091E8009E779093E80018
:101B9000E0920001882329F2CF70C093E90080E031
:101BA000DF91CF911F910F91FF90EF900895E091F9
:101BB000030177CF9091C1028091C202891751F041
:101BC000E92FF0E0EF53FE4F80819F5F9093C102B9
:101BD00090E008958FEF9FEF08958330C9F128F4C6
:101BE000813061F0823019F10895853009F452C0D6
:101BF00008F43FC0863009F45EC008958091170153
:101C0000681790F4861B80931701809117011F922B
:101C10008F938AEF97E09F938F930E949B050F907D
:101C20000F900F900F90089510921701EECF8091B2
:101C30001601681750F4861B8093160180911601D7
:101C40001F928F9388EE97E0E6CF10921601F6CFA1
:101C500080911501681750F4861B809315018091BF
:101C600015011F928F9385ED97E0D5CF1092150146
:101C7000F6CF80911401681750F4861B80931401ED
:101C8000809114011F928F9380EC97E0C4CF109243
:101C90001401F6CF80911301681750F4861B8093CE
:101CA0001301809113011F928F9387EA97E0B3CFBE
:101CB00010921301F6CF80911201681750F4861B21
:101CC00080931201809112011F928F938CE897E00C
:101CD000A2CF10921201F6CF833009F445C028F448
:101CE000813061F0823049F10895853009F46AC08D
:101CF00008F451C0863009F47CC008958091170122
:101D0000482F460F5527551F4F3F510594F4680F34
:101D100060931701809117011F928F938DE797E0D1
:101D20009F938F930E949B050F900F900F900F90A1
:101D300008958FEF80931701EDCF80911601482F02
:101D4000460F5527551F4F3F510554F4680F6093B8
:101D50001601809116011F928F938BE697E0E0CFDA
:101D60008FEF80931601F5CF80911501482F460F14
:101D70005527551F4F3F510554F4680F60931501C7
:101D8000809115011F928F9388E597E0C9CF8FEF5F
:101D900080931501F5CF80911401482F460F5527E8
:101DA000551F4F3F510554F4680F60931401809103
:101DB00014011F928F9383E497E0B2CF8FEF80934B
:101DC0001401F5CF80911301482F460F5527551F59
:101DD0004F3F510554F4680F609313018091130134
:101DE0001F928F938AE297E09BCF8FEF809313012E
:101DF000F5CF80911201482F460F5527551F4F3FB1
:101E0000510554F4680F60931201809112011F92E2
:101E10008F938FE097E084CF8FEF80931201F5CFFF
:101E2000CF93DF93209101033091020328173907E4
:101E300001F19093020380930103E091C603F091B6
:101E4000C7033097B1F0EC010084F185E02D0995CE
:101E50008091D5038570853061F4DF93CF9385E859
:101E600092E09F938F930E949B050F900F900F908D
:101E70000F90DF91CF910895CF93DF932091FF02D0
:101E8000309100032817390701F1909300038093E4
:101E9000FF02E091C603F091C7033097B1F0EC0167
:101EA0000680F781E02D09958091D50385708530F6
:101EB00061F4DF93CF9387E792E09F938F930E9423
:101EC0009B050F900F900F900F90DF91CF91089589
:101ED00087E598E00E9402051F9281E08F931F9290
:101EE00085E08F9389E098E09F938F930E949B05F4
:101EF0000F900F900F900F900F900F900895CF9329
:101F00008091D50383FF7EC081E194E00E940205A9
:101F10008091CA031F928F938CE094E09F938F93DC
:101F20000E949B058AE094E00E9402058091CB0309
:101F3000282F082E000C330B3F938F9387E094E0FB
:101F40009F938F930E949B0585E094E00E94020579
:101F50008091CC03282F082E000C330B3F938F93D6
:101F600082E094E09F938F930E949B0580E094E031
:101F70000E9402058091CD03282F082E000C330B00
:101F80003F938F938DEF93E09F938F930E949B05D8
:101F90008BEF93E00E9402058091CE03282F082E3C
:101FA000000C330B3F938F9388EF93E09F938F93B5
:101FB0000E949B0585EF93E00E9402058091C50376
:101FC0001F928F9382EF93E09F938F930E949B05C4
:101FD00080EF93E00E9402058091C4031F928F93CB
:101FE0008DEE93E09F938F930E949B058AEE93E082
:101FF0000E9402058DB79EB74C960FB6F8949EBF0F
:102000000FBE8DBFE091C603F091C7033097F1F189
:10201000C091CA030480F581E02D8AEC93E0099514
:10202000C093CA038091D50383FF30C08091CE0353
:10203000282F082E000C330B3F938F938091CD03F4
:10204000282F082E000C330B3F938F938091CC03E5
:10205000282F082E000C330B3F938F938091CB03D6
:10206000282F082E000C330B3F938F931F92CF9392
:1020700084E394E09F938F930E949B058DB79EB756
:102080000C960FB6F8949EBF0FBE8DBF0E943F07FF
:102090009093C9038093C803CF9108950F931F9322
:1020A000CF93DF938091C2039091C103892B8093DA
:1020B000B4019091C003992389F0892B8093B401D6
:1020C000E5EBF1E02CEB31E080E0919191118F5F35
:1020D0002E173F07D1F781111092C003E091C6037C
:1020E000F091C7033097B1F10280F381E02D84EBCA
:1020F00091E009958091D50382FF2CC080FF04C038
:102100008FE593E00E940205D0E0C0E009E513E00E
:102110008091D50380FF0EC0FE01EC54FE4F8081FC
:102120001F928F931F930F930E949B050F900F9008
:102130000F900F902196C830D10551F78091D503AB
:1021400080FF08C087E593E0DF91CF911F910F9149
:102150000C940205DF91CF911F910F910895109279
:10216000C2031092C103E4EBF1E0118212821382E8
:1021700014821582168217820E944E1085E0EAECC6
:10218000F3E0DF011D928A95E9F71092C5031092E2
:10219000C4030E947F0F90E080E00E943C0F90E01B
:1021A00080E00C94100FCF93C82F1F928F9382E57D
:1021B00099E09F938F930E949B0581E090E0A0E0BF
:1021C000B0E004C0880F991FAA1FBB1FCA95D2F7A1
:1021D0008093D6039093D703A093D803B093D903E9
:1021E0000F900F900F900F90CF910C94AF10882309
:1021F00041F080959091C20389238093C2030C948F
:102200004E100895882339F09091C203892B809352
:10221000C2030C944E1008958823E1F19CEF980FAF
:10222000913A68F4E4EBF1E09281891301C01282E3
:10223000319641E0EA3BF407B9F70C944E1090E276
:10224000980F983088F4877021E030E0A90102C02F
:10225000440F551F8A95E2F7CA0180959091C203F9
:1022600089238093C203E9CF9BE5980F933020F434
:1022700090E080E00C943C0F98E5980F973120F4A3
:1022800090E080E00C94100F803F20F00E94A405A5
:102290000C947F0F08958732D8F58E3108F0FCC07A
:1022A0008E3009F48FC078F4873009F470C08B3019
:1022B00009F456C0863009F458C089E095E00E94C0
:1022C000020580E00895863109F4A6C078F48031D3
:1022D000A1F79091D503892F877F93FF8860809322
:1022E000D50383FF7FC08BE996E063C0893109F491
:1022F0007CC08B3111F79091D503892F8D7F91FF91
:1023000082608093D50381FF5AC084ED96E051C06E
:10231000883331F150F4893221F0853311F087325E
:1023200061F680E00E94D31040C08334D1F320F4E2
:102330008A3318F28953F6CF883409F0BECF0E9451
:10234000AF108AEF96E00E9402052FEF83ED90E335
:10235000215080409040E1F700C000000E94B10889
:102360008FE494E00E94020520C08091D503817F14
:102370008E7F8093D50382EE94E00E9402058BE06D
:1023800097E00E94020581E08093D4030895809134
:10239000D50380FF0CC08DEE96E00E94020580916F
:1023A000D503817F8E7F8093D50381E0089581EEF0
:1023B00096E00E9402058091D5038160F4CF86ECFF
:1023C00096E0D0CF9091D503892F8B7F92FF8460C8
:1023D0008093D50382FF03C087EB96E0EACF87EABC
:1023E00096E0C0CF8EE896E0BDCF8FE796E00E94E2
:1023F000020583E596E00E9402058BE096E00E94CC
:10240000020585EE95E00E94020580EA95E00E94B3
:10241000020584E795E0A6CF86E695E00E940205D6
:102420000E948E081F928F938CE495E09F938F9368
:102430000E949B05809111011F928F9385E395E087
:102440009F938F930E949B058091D3031F928F933C
:1024500082E295E09F938F930E949B052FB7F8949B
:102460008091CF039091D003A091D103B091D2037A
:102470002FBFBF93AF939F938F938BE095E09F9374
:102480008F930E949B058DB79EB742960FB6F89426
:102490009EBF0FBE8DBF89CF8D5144CFCF93882370
:1024A00009F4ABC0C82F8CEF8C0F813A08F051C1F2
:1024B0008091D403813059F1F8F0823009F455C08D
:1024C0001092D403A6EBB1E0EFEF80E09D91C91725
:1024D00081F0EF3F19F4911101C0E82F8F5F863032
:1024E000A9F7EF3F31F00E2E000CFF0BEC54FE4F1E
:1024F000C283CF910C944E108091B40181528230EE
:1025000008F78C2F0E944B11811177C0DBCF80918F
:10251000B40181528230A8F3C431C9F048F4CB3001
:1025200059F0C031C1F085E992E00E94020511C066
:10253000C93269F0C833B9F782EE94E00E9402050F
:102540008BE992E00E94020581E08170DDCF10925C
:10255000D40380E0FACF0E94680F87E992E00E94DE
:10256000020582E08093D403EFCFC432C8F4CE31A9
:1025700008F0BEC0CB30E1F040F4C73009F4CFC062
:1025800084E493E0CF910C940205C331C1F1C431CE
:10259000B9F780910303882349F1109203030AC01D
:1025A000CB3409F4BAC0C0F4C93299F3C83341F747
:1025B0000E94680F80910303882309F4C7C01F920B
:1025C0008F938EE393E09F938F930E949B050F90D0
:1025D0000F900F900F9011C0C13509F498C0C2350B
:1025E00009F48FC0CE3461F66AE092C083E593E0CF
:1025F0000E94020581E08093D403CF9108958DE27B
:1026000093E00E9402058BE193E00E940205809115
:1026100017011F928F9388E193E09F938F930E94FD
:102620009B0586E193E00E94020584E093E00E940E
:102630000205809116011F928F9381E093E09F9392
:102640008F930E949B058FEF92E00E94020580EF1E
:1026500092E00E940205809115011F928F938DEEEA
:1026600092E09F938F930E949B058BEE92E00E94D5
:1026700002058AED92E00E940205809114011F92EA
:102680008F9387ED92E09F938F930E949B0585ED3A
:1026900092E00E94020580EC92E00E940205809187
:1026A00013011F928F938DEB92E09F938F930E9463
:1026B0009B058BEB92E00E94020584EA92E00E9467
:1026C0000205809112011F928F9381EA92E09F93FD
:1026D0008F930E949B058FE992E00E9402058DB7BF
:1026E0009EB748960FB6F8949EBF0FBE8DBF62CFBF
:1026F000CE51EC2FF0E0E85DFE4F80818093030324
:1027000059CF61E0809103030E946C0E53CF61E0CA
:10271000809103030E94ED0D4DCF6AE0F3CF8EE16F
:102720008093170182E3809316018AE0809315015C
:1027300084E18093140188E08093130188E2809300
:10274000120186E493E00E94020534CF8BE393E00C
:1027500019CF80E28C0F883068F4C77021E030E038
:1027600001C0220FCA95EAF78091C203822B8093A1
:10277000C203BFCE8BE58C0F833068F481E890E014
:10278000C53A31F083E890E0C63A11F482E890E06F
:10279000CF910C943C0F88E58C0F873108F068C00E
:1027A00082EE90E0C83A09F460C089EE90E0C93A40
:1027B00009F45BC08AEE90E0CA3A09F456C085EB92
:1027C00090E0CB3A09F451C086EB90E0CC3A09F4A2
:1027D0004CC083EB90E0CD3A09F447C084EB90E025
:1027E000CE3A09F442C087EB90E0CF3AF1F18CEC9D
:1027F00090E0C13BD1F18DEC90E0C03BB1F183E8BA
:1028000091E0C23B91F18AE891E0C33B71F182E92A
:1028100091E0C43B51F184E991E0C53B31F181E2A3
:1028200092E0C63B11F183E292E0C73BF1F084E213
:1028300092E0C83BD1F085E292E0C93BB1F086E27C
:1028400092E0CA3B91F087E292E0CB3B71F08AE2E2
:1028500092E0CC3B51F08FE690E0CD3B31F090E040
:1028600080E0CE3B11F480E790E0CF910C94100F04
:10287000CF3B69F40E94AF109FEF20E782E09150B8
:1028800020408040E1F700C000000E94B108C03F36
:1028900008F4B3CE8C2F0E94AF06CF910C947F0F1B
:1028A000CF92DF92EF92FF920F931F93CF93DF931C
:1028B00000D000D01F92CDB7DEB76C0185E0F601E5
:1028C000DE01119601900D928A95E1F7F6014081A3
:1028D00051812381348191E02115310531F05F3F31
:1028E00019F491E04F3F09F090E090FD99C0F60196
:1028F0000281F580F2949FE0F92249835A830B8389
:10290000722F3D832C83602F8D810E944B07182FDF
:10291000E92FE295EF70EF3008F082C0F0E0ED565D
:10292000FB4E0C943321A214A214E014E0145615AB
:102930008815101510159E1510157416741610159F
:1029400010153017F92FFF70FF2E907F19F0F294B9
:1029500080EFF8220023C9F0FF2039F08091C103F5
:10296000F82AF092C1030E944E10812F0F900F9011
:102970000F900F900F90DF91CF911F910F91FF90CB
:10298000EF90DF90CF900C944E12812F0E940C118B
:10299000FF2009F445C0F0948091C103F822F09221
:1029A000C1030F900F900F900F900F90DF91CF9178
:1029B0001F910F91FF90EF90DF90CF900C944E10ED
:1029C000892F8F70907F903211F08295807F112334
:1029D00079F0113009F449C0002309F455C0FF20F3
:1029E00059F0F601958190FF8DC19F70958304C0C9
:1029F000002321F1F1100FC00F900F900F900F9056
:102A00000F90DF91CF911F910F91FF90EF90DF908A
:102A1000CF900C94021121E0F212EECF8093C0030C
:102A20000F900F900F900F900F90DF91CF911F910B
:102A30000F91FF90EF90DF90CF900895F11011C0AB
:102A40001092C0030F900F900F900F900F90DF9196
:102A5000CF911F910F91FF90EF90DF90CF900C944A
:102A6000F71091E0F912ECCFDBCF002349F0E5E05D
:102A7000EF15B0F29091C203982309F4BDCFE2CFD5
:102A8000F4E0FF1568F2DECFFF20E1F2812F0F9016
:102A90000F900F900F900F90DF91CF911F910F919A
:102AA000FF90EF90DF90CF900C940C11892F8695BA
:102AB00086958370C1F0813009F0B2CF812F937079
:102AC000011102C090E080E00F900F900F900F90E6
:102AD0000F90DF91CF911F910F91FF90EF90DF90BA
:102AE000CF900C94100F812F9370011102C090E0D1
:102AF00080E00F900F900F900F900F90DF91CF918B
:102B00001F910F91FF90EF90DF90CF900C943C0FAE
:102B1000002389F00E94AF060F900F900F900F9046
:102B20000F90DF91CF911F910F91FF90EF90DF9069
:102B3000CF900C947F0F0E94A405EECF892F837055
:102B400009F064C001116CCF812F82958695877042
:102B5000880F880F412F4F70C42ED12CF12CE12CFF
:102B6000082E04C0CC0CDD1CEE1CFF1C0A94D2F70E
:102B700040E050E0BA0114FF11C00FE010E020E087
:102B800030E004C0000F111F221F331F8A95D2F7B7
:102B9000B901A80140955095609570950091D603B4
:102BA0001091D7032091D8033091D903969596952B
:102BB00093709230E9F028F5913089F04C295D2925
:102BC0006E297F2940235123622373234093D60328
:102BD0005093D7036093D8037093D90321CFC02AB1
:102BE000D12AE22AF32A4C295D296E297F29EECFCA
:102BF0004C295D296E297F29402751276227732799
:102C0000E5CF4023512362237323EDCF8695002324
:102C100011F0892F8170882309F402CF812F8295CA
:102C200086958770880F880F412F4F70C42ED12C46
:102C3000F12CE12C082E04C0CC0CDD1CEE1CFF1C7A
:102C40000A94D2F740E050E0BA0114FF11C00FE03F
:102C500010E020E030E004C0000F111F221F331FDE
:102C60008A95D2F7B901A801409550956095709565
:102C700000913C0310913D0320913E0330913F03AE
:102C80009695969593709230E9F028F5913089F0F9
:102C90004C295D296E297F29402351236223732308
:102CA00040933C0350933D0360933E0370933F0376
:102CB000B7CE0C291D292E293F29402B512B622BE1
:102CC000732BEECF4C295D296E297F294027512790
:102CD00062277327E5CF40235123622373234C29B6
:102CE0005D296E297F29DCCF803F09F44EC0D0F4E6
:102CF00080E4810F803270F1002309F4ACC0FF2022
:102D000009F4A6C0812F0E944E12193309F099C010
:102D1000FFEF21EE84E0F15020408040E1F700C059
:102D200000007ECE823F09F470C008F45BC0833F90
:102D300019F7002309F47CC0292F2F7181E090E05E
:102D4000A0E0B0E004C0880F991FAA1FBB1F2A95FE
:102D5000D2F73AC0E12FE071FE2E892F8F71002348
:102D600051F00E941808812F8295807FF11044CE87
:102D7000812F8F7041CE0E94F407812F8295807F32
:102D8000F11060CE812F8F705DCE002331F1F4E021
:102D9000FF1508F445CE292F2F7181E090E0A0E0C7
:102DA000B0E004C0880F991FAA1FBB1F2A95D2F755
:102DB00040913C0350913D0360913E0370913F036D
:102DC00084279527A627B72780933C0390933D033C
:102DD000A0933E03B0933F0323CE25E02F1508F4C4
:102DE0001FCED9CF892F8F71002399F00F900F90AC
:102DF0000F900F900F90DF91CF911F910F91FF9047
:102E0000EF90DF90CF900C941808892F8F710023DA
:102E100069F30F900F900F900F900F90DF91CF916B
:102E20001F910F91FF90EF90DF90CF900C94F407DB
:102E300010923C0310923D0310923E0310923F0308
:102E4000EFCD133509F464CF173409F0E9CD60CF25
:102E5000892F8F71CBCFF11019CE892F8F71D9CFD8
:102E60008111DECD002309F4DBCD0E94AF108FEF7E
:102E700090E7E2E081509040E040E1F700C00000C0
:102E80000E94B1081F93CF93DF9380910903807F45
:102E9000B1F480910603882391F020913B031091B7
:102EA0000A03C0910403D0910503A0910703B091D8
:102EB000080341E0CF3F09F040E0121304C0DF9166
:102EC000CF911F91089581E0109721F0842FDF3F6B
:102ED00009F080E030E080FD33C0C90166E070E0B9
:102EE0000E940E21FC01E55FFC4F81818D1328C0FB
:102EF00080818C1325C08281811122C083819481BD
:102F00008A1B9B0B883C9105D8F4809109038F7034
:102F1000806180930903C90166E070E00E940E2180
:102F2000FC01E05FFC4F90819F709061908384E092
:102F300093E00E945014DF91CF911F910C943808B8
:102F40002F5F3F4F2770B9CF9F92AF92BF92CF9222
:102F5000DF92EF92FF920F931F93CF93DF93CDB742
:102F6000DEB761970FB6F894DEBF0FBECDBF8C0100
:102F700085E0F801DE011D9601900D928A95E1F73A
:102F8000F80140812181F280C380D48090910403B4
:102F900030910503609107037091080381E061158A
:102FA000710531F03F3F19F481E09F3F09F080E067
:102FB000F82FF1709F2E80FD4EC184E0A82E83E093
:102FC000B82EE0900603F601E61BF70BEE2009F49D
:102FD00004C180910903582F507FE83CF10508F0A7
:102FE000BDC0511183C0EF2C321322C0941320C0F6
:102FF000F1101EC08F70806180930903C5010E948B
:10300000501480910903F80185838E2D61960FB6C7
:10301000F894DEBF0FBECDBFDF91CF911F910F910E
:10302000FF90EF90DF90CF90BF90AF909F9008956A
:1030300081E0C114D10431F02F3F19F481E04F3FFA
:1030400009F080E080FD14C081E08F25F82FF17039
:10305000BF2EE0913B0330910A0380FD22C0FF2088
:10306000A1F280910903816080930903E12CCDCF07
:1030700080E0ECCFF0E0CF0166E070E00E940E212E
:10308000DC01A55FBC4F11968C911197281307C0E6
:103090008C91481304C012968C918F11E0CF319619
:1030A000E770E313E7CF7C2DD98AC88A522F6F2DA2
:1030B00089890E944B07292F22952F70223050F0CA
:1030C000243078F49F7051F0F8019581907F31F4AD
:1030D000E92C9BCF9F7011F08823D1F3805E88305C
:1030E000B8F3C8010E9450149B2CF2CF321306C0D3
:1030F000941304C0F801FF2009F48AC04D872E877D
:10310000FF867C2DD98AC88A522F6F2D89890E940B
:103110004208882309F4AEC0FF2009F4ABC08091B7
:103120000903803270F02091040330910503388741
:103130002F831986DB86CA868C87CE0107960E946C
:10314000501486E0F801A4E0B3E001900D928A9556
:10315000E1F70E944217EE24E39457CF51110AC0C1
:1031600084E093E00E94501486E0F50111928A9564
:10317000E9F77CCF32130FC094130DC0F1100BC0D0
:10318000F8018583C8010E94501486E0F501119270
:103190008A95E9F73ACF4D872E87FF867C2DD98A0D
:1031A000C88A522F6F2D89890E944208882309F40A
:1031B00061C0FF2009F45EC080910903803208F2EB
:1031C00020910403309105033A8329831B82DD8219
:1031D000CC828E83CE010196B2CFE83CF105A8F6F1
:1031E000EF2CFF2009F446C032131FC094131DC0FA
:1031F0008091090380FD10C0982F907F69F0F8013D
:103200008583903F31F0982F907F905F8F70892B4E
:103210008583C8010E94501486E0F801A4E0B3E061
:1032200001900D928A95E1F7F0CE4D872E87FF86AB
:103230007C2DD98AC88A522F6F2D89890E94420815
:1032400081117FCF80910903816080930903C801B8
:103250000E945014DACEFF2069F04D872E87FF863A
:103260007C2DD98AC88A522F6F2D89890E944208E5
:10327000811167CFC8010E9450146DCFCF93DF93A7
:10328000CDB7DEB767970FB6F894DEBF0FBECDBFE0
:103290004B8B5C8B6D8B7E8B8F8B1A8A198A85E0AA
:1032A000FE017396DE011D9601900D928A95E1F75D
:1032B00086E0FE013D96DE01179601900D928A95FB
:1032C000E1F7CE0107960E94A417811138C086E06D
:1032D000FE013796DE01119601900D928A95E1F775
:1032E0009F8188852A853B85232B39F08F3F19F4F0
:1032F00081E09F3F19F080E001C081E080FD1FC0A8
:1033000080910A0390E09C012F5F3F4F2770332785
:1033100040913B034217130661F166E070E00E94A2
:103320000E21DC01A55FBC4F96E0FE0131960190B5
:103330000D929A95E1F720930A030E943808809134
:103340003B0390910A03891709F190E066E070E071
:103350000E940E21855F9C4F0E94A4178823B1F024
:1033600080913B0390E001968770992780933B03FF
:10337000E6CF0E94AF1010920A0310923B0386E042
:10338000E4E0F3E0DF011D928A95E9F767960FB656
:10339000F894DEBF0FBECDBFDF91CF910895CF93DC
:1033A000DF9300D01F92CDB7DEB72091FE0224300C
:1033B00041F520911001222321F123E029839B83F1
:1033C0008A8382E08093E9008FEF9091E80081503A
:1033D00095FD06C095ED9A95F1F700008111F5CFA6
:1033E0008091E80085FF0DC050E040E063E070E0B0
:1033F000CE0101960E94AA0C8091E8008E778093FE
:10340000E8000F900F900F90DF91CF910895CF9328
:10341000DF9300D01F92CDB7DEB72091FE0224309B
:1034200081F520911001222361F119821A821B82F9
:1034300022E029838138910520F0805891099B83EF
:103440008A8382E08093E9008FEF9091E8008150B9
:1034500095FD06C095ED9A95F1F700008111F5CF25
:103460008091E80085FF0DC050E040E063E070E02F
:10347000CE0101960E94AA0C8091E8008E7780937D
:10348000E8000F900F900F90DF91CF910895209159
:10349000FE02243049F522E02093E9002FEF30911D
:1034A000E800215035FD06C035ED3A95F1F70000F2
:1034B0002111F5CF2091E80025FF16C020911001C1
:1034C00050E040E063E070E0222339F021E02093F7
:1034D000F10050E040E065E070E00E94AA0C8091AD
:1034E000E8008E778093E8000895CF93DF932091D2
:1034F000FE02243011F521E02093E90021E821505B
:1035000021F03091E80035FF1BC02091E80025FF35
:1035100014C0EC0150E040E068E070E00E94AA0CAA
:103520008091E8008E778093E80088E0FE01ABEEA2
:10353000B2E001900D928A95E1F7DF91CF91089565
:10354000EFE3F1E03197F1F700C00000D8CFEF9240
:10355000FF920F931F93CF93DF93C82F1F928F93E8
:103560008EE591E09F938F930E949B050F900F90A3
:103570000F900F908091C80085FFFCCFC093CE00C4
:103580008FE39CE90197F1F700C0000010E000E034
:1035900087E5E82E81E0F82E0E94DA0DEC01CF3F9E
:1035A000DC0719F48FEF9FEF1EC0CE018F778B37AA
:1035B000910519F08C2F902F8C01DF93CF93FF9200
:1035C000EF920E949B050F900F900F900F90CB3FB2
:1035D000D10511F785E591E09F938F930E949B059C
:1035E000C8010F900F90DF91CF911F910F91FF9025
:1035F000EF900895CF93DF930E94DA0DEC01CF3F57
:10360000DC0799F49091D4028091BC01981759F08D
:1036100080EB0E94A71A8091D4020E94A71A809181
:10362000D4028093BC0180E039C0DF93CF9385E65C
:1036300091E09F938F930E949B058C2F9E0193E0B6
:10364000359527959A95E1F79C2F977061E070E08A
:10365000DB0102C0AA0FBB1F9A95E2F7E22FEF70C1
:10366000F0E00F900F900F900F90EC53FD4F4081C2
:1036700050E04A235B23C7FF14C0452B79F02F701D
:103680003327F901EC53FD4FC770DD2701C0660FEA
:10369000CA95EAF76095908169236083DF91CF91A5
:1036A0000895452BD9F72F703327F901EC53FD4FBF
:1036B000C770DD2701C0660FCA95EAF79081692BB4
:1036C000ECCF78941F920F920FB60F9211248F9324
:1036D0009F93AF93BF938091CF039091D003A0911C
:1036E000D103B091D2030196A11DB11D8093CF03E8
:1036F0009093D003A093D103B093D203BF91AF9125
:103700009F918F910F900FBE0F901F9018951F9251
:103710000F920FB60F9211248F939F93AF93BF9385
:103720008091C303811113C08091CF039091D00386
:10373000A091D103B091D2034196A11DB11D8093F8
:10374000CF039093D003A093D103B093D203BF9142
:10375000AF919F918F910F900FBE0F901F90189572
:103760001F920F920FB60F9211242F933F934F93F6
:103770005F936F937F938F939F93AF93BF93EF93D9
:10378000FF938091E10082FF09C08091E20082FFF7
:1037900005C08091E1008B7F8093E1008091E10082
:1037A00080FF1FC08091E20080FF1BC08091E2007B
:1037B0008E7F8093E2008091E20080618093E2003E
:1037C0008091D80080628093D80019BC85E08093F6
:1037D000FE028091EA028093E9021092EA020E94BE
:1037E000AF108091E10084FF2DC08091E20084FF42
:1037F00029C084E089BD86E089BD09B400FEFDCF03
:103800008091D8008F7D8093D8008091E1008F7ED9
:103810008093E1008091E2008F7E8093E2008091AE
:10382000E20081608093E2008091F502882309F430
:103830005EC084E08093FE020E94AF108091E90296
:103840008093EA028091E10083FF40C08091E20012
:1038500083FF3CC08091E100877F8093E10082E09C
:103860008093FE021092F5028091E1008E7F80939A
:10387000E1008091E2008E7F8093E2008091E2007F
:1038800080618093E20042E060E080E00E947A097B
:1038900081E0809311011092D3031092EA0298E024
:1038A000EBEEF2E0DF011D929A95E9F71092B50177
:1038B0001092B6011092B7011092B8011092B9019E
:1038C0001092BA011092BB0180931001FF91EF9109
:1038D000BF91AF919F918F917F916F915F914F9128
:1038E0003F912F910F900FBE0F901F9018958091D0
:1038F000E30087FD02C081E09DCF83E09BCFCF93A3
:10390000DF93CDB7DEB72C970FB6F894DEBF0FBEAE
:10391000CDBF84B7877F84BF0FB6F894A8958091F8
:103920006000886180936000109260000FBE80E8A4
:1039300090E00FB6F89480936100909361000FBE01
:1039400081EF9CE0909333018093320186E091E017
:103950009093C7038093C6038EEA91E00E9402050C
:103960000E949A08809163008E7F8093630081E0BB
:103970008093E8021092E2001092E1008091D8005A
:103980008F778093D8008091D80080688093D8008A
:103990008091D8008F7D8093D80084E089BD86E037
:1039A00089BD09B400FEFDCF1092FE021092F5020F
:1039B0001092F4021092F30242E060E080E00E9474
:1039C0007A098091E1008E7F8093E1008091E2008E
:1039D00081608093E2008091E20088608093E20041
:1039E0008091E0008E7F8093E000789482E084BD37
:1039F00093E095BD9AEF97BD80936E0087E6809324
:103A0000CC001092CD008091C90088698093C900D4
:103A1000789484ED92E0B4ECCB2EB2E0DB2EF6018C
:103A200011926F018E179F07D1F78091FE028430AB
:103A300009F042C10E94D90C882309F43DC18CE9E8
:103A400091E00E94020580E80E94A71A82E80E9485
:103A5000A71A81E80E94A71A83E80E94A71A8EE895
:103A600091E00E940205F3E84F2EF1E05F2EA8E1FD
:103A70006A2E712C8091FE02853009F420C10E94CB
:103A8000FA1A06ED12E0E4ECAE2EE2E0BE2E312C86
:103A9000F50121905F01F8019080921409F468C04B
:103AA0008091D50381FF40C086E791E00E94020526
:103AB00024EC32E03C872B87F12CE12CEB85FC8554
:103AC0002191FC87EB87229530E0C901880F991F6F
:103AD000880F991F8C7C35952795359527952373ED
:103AE000822B90E028E131E03F932F939C01220F3D
:103AF000331F2A7A959587958575822B1F928F9310
:103B0000FF92EF928BE691E09F938F930E949B052B
:103B1000FFEFEF1AFF0A0FB6F894DEBF0FBECDBF5E
:103B200030E1E316F10451F6E12CFF24F3949224E2
:103B3000892D8F21C1F0EE823F8291E08F2D82216D
:103B400009F490E098870E943F078160782F9A8758
:103B500089874E815F8168858A850E943E19F801B8
:103B600080818F258083E394FF0CF8E0EF12E0CF93
:103B700033940F5F1F4F20E132128ACF3FEF39831A
:103B80003A831B820E943F078160782F9D838C833C
:103B900049815A816B818D810E943E198091C803B1
:103BA0009091C9032FB7F8944091CF035091D0035F
:103BB0006091D1037091D2032FBFFA01E81BF90B7A
:103BC0002091C5038091160190E0211107C08091DA
:103BD000170190E06AE070E00E940E21E817F907F3
:103BE00080F08091CB03F090CC031091CD03009135
:103BF000CE0381119AC0F1105EC111115CC1011197
:103C00005AC10E948E089091D502891701F10E9435
:103C10008E088093D5029091D5039570953051F41C
:103C20001F928F935F924F920E949B050F900F906F
:103C30000F900F908091D50281FDE5C01092D402C3
:103C400080FF05C08091D40288608093D4022091C7
:103C5000E4003091E5008091E6029091E702281798
:103C6000390739F18091E4009091E5009093E702E3
:103C70008093E6020E94D90C8823D9F08091FE023D
:103C80008430B9F48091E9008F709091EC0090FF3E
:103C9000BEC090E8892B93E09093E9009091EB00EF
:103CA00090FF04C09091EE0097FDCFC08F7080937D
:103CB000E9000E94AC09DECE0E94AC09B6CE80912C
:103CC000FE02843011F11092C30380E40FB6F89421
:103CD000A895609260000FBE8093600083B7817FDB
:103CE000846083BF83B7816083BF7894889583B7EE
:103CF0008E7F83BF0FB6F894A8958091600088618D
:103D000080936000109260000FBE8091F4028823BF
:103D100009F4B0CE0E94FA1AE4ECF2E0819181112C
:103D2000B4C0CE16DF06D1F7A5CE2F3F19F02F5F16
:103D30002093C503181624F40E9463068093CB03D6
:103D40008091CB0387FF05C00E9463068195809315
:103D5000CB031F1424F40E9463068093CC0380914C
:103D6000CC0387FF05C00E94630681958093CC0336
:103D70006091CB03662331F1F090CC03FF2011F169
:103D8000062E000C770B880B990B0E940D2023E365
:103D900033E343E35FE30E9471200E94D51F6093E9
:103DA000CB036F2DFF0C770B880B990B0E940D2016
:103DB00023E333E343E35FE30E9471200E94D51FB6
:103DC0006093CC03111624F40E9428068093CD033F
:103DD0008091CD0387FF05C00E94280681958093BE
:103DE000CD03101624F40E9428068093CE03809100
:103DF000CE0387FF05C00E94280681958093CE03DD
:103E00000E947F0FFECE94E09093D40219CF90E0F1
:103E100041CFE0910101F0910201E90FF11D2081F4
:103E20009F5F309105019323909304012093F1004B
:103E30009091E80095FD09C09091E80090FF05C0C1
:103E40009091E8009E779093E80090910401209172
:103E50000301291721F02091E80025FDDACF909188
:103E6000F200992309F422CF9091E80090FF1ECF31
:103E70009091E80095FD06C09091E8009E779093A0
:103E8000E80014CF1092F100F3CF84E089BD86E002
:103E900089BD09B400FEFDCF8091D8008F7D80934D
:103EA000D8008091E00082608093E0008091E00083
:103EB00081FDFCCFDFCD2F3F09F039CF4ACF1F92D4
:103EC0000F920FB60F9211248F939F93EF93FF934E
:103ED0008091C202E82FF0E08F5F9091C1029817A5
:103EE00039F09091CE00EF53FE4F90838093C20241
:103EF000FF91EF919F918F910F900FBE0F901F90A8
:103F000018951F920F920FB60F9211248F939F93C3
:103F1000AF93BF938091BD019091BE01A091BF016D
:103F2000B091C001892B8A2B8B2B69F18BB192E068
:103F300089278BB98091BD019091BE01A091BF01ED
:103F4000B091C001181619061A061B069CF4809140
:103F5000BD019091BE01A091BF01B091C001019738
:103F6000A109B1098093BD019093BE01A093BF0147
:103F7000B093C001BF91AF919F918F910F900FBEF1
:103F80000F901F90189580916F008D7F80936F0028
:103F900010928000109281008FB7F89410928900DF
:103FA000109288008FBF5998E5CF0E94DC1F68945B
:103FB000B1110C946B2008950E94502088F09F57F7
:103FC00098F0B92F9927B751B0F0E1F0660F771F3D
:103FD000881F991F1AF0BA95C9F714C0B13091F033
:103FE0000E946A20B1E008950C946A20672F782F10
:103FF0008827B85F39F0B93FCCF3869577956795F8
:10400000B395D9F73EF490958095709561957F4F63
:104010008F4F9F4F0895E89409C097FB3EF4909509
:104020008095709561957F4F8F4F9F4F9923A9F091
:10403000F92F96E9BB279395F69587957795679520
:10404000B795F111F8CFFAF4BB0F11F460FF1BC064
:104050006F5F7F4F8F4F9F4F16C0882311F096E9F7
:1040600011C0772321F09EE8872F762F05C06623A5
:1040700071F096E8862F70E060E02AF09A95660F5E
:10408000771F881FDAF7880F9695879597F9089517
:1040900057FD9058440F551F59F05F3F71F04795F9
:1040A000880F97FB991F61F09F3F79F087950895DE
:1040B000121613061406551FF2CF4695F1DF08C0FD
:1040C000161617061806991FF1CF8695710561051A
:1040D00008940895E894BB2766277727CB0197F9C2
:1040E00008950E9483200C94FD200E94EF2038F058
:1040F0000E94F62020F0952311F00C94E6200C94F9
:10410000EC200C946B200E94482078F39923C9F38B
:104110005523B9F3950F50E0551FAA27EE27FF2727
:10412000BB2700240894679520F4E20FF31FB41F07
:104130000A1E220F331F441FAA1F6695A9F7779501
:1041400030F4F30FB41F0A1E121E08F46395330FE8
:10415000441FAA1F221F769599F7879520F4B40F64
:104160000A1E121E631F440FAA1F221F331F8695AB
:10417000A9F7862F712D602D11249F5750409AF07A
:10418000F1F088234AF0EE0FFF1FBB1F661F771F59
:10419000881F91505040A9F79E3F510580F00C9424
:1041A000E6200C946B205F3FE4F3983ED4F38695B1
:1041B00077956795B795F795E7959F5FC1F7FE2BC4
:1041C000880F911D9695879597F9089597F99F67A0
:1041D00080E870E060E008959FEF80EC089500248F
:1041E0000A941616170618060906089500240A945C
:1041F00012161306140605060895092E0394000CE2
:1042000011F4882352F0BB0F40F4BF2B11F460FF70
:1042100004C06F5F7F4F8F4F9F4F08950024552735
:1042200004C0080E591F880F991F009729F0769532
:104230006795B8F37105B9F7802D952F089597FB11
:10424000072E16F4009407D077FD09D00E9439217B
:1042500007FC05D03EF4909581959F4F0895709589
:1042600061957F4F0895EE0FFF1F0590F491E02DAB
:104270000994AA1BBB1B51E107C0AA1FBB1FA617AD
:10428000B70710F0A61BB70B881F991F5A95A9F7FF
:0E42900080959095BC01CD010895F894FFCF64
:10429E0005340100007FD60C751A471A071ACF197C
:1042AE0001012808140A321E00407F2215019600D3
:1042BE007400D901F2010B0201020304050607087E
:0242CE000900E5
:106800005300EA44E9448140040005000600070003
:10681000080009000A000B000C000D000E000F001C
:1068200010001100120013001400150016001700CC
:10683000180019001A001B001C001D001E001F007C
:10684000200021002200230024002500260027002C
:10685000280029002A002B002C002D002E002F00DC
:106860003000310035003300340035003600370089
:10687000380039003A003B003C003D003E003F003C
:1068800040004100420043004400450046004700EC
:10689000480049004A004B004C004D004E004F009C
:1068A000500051005200530054005500560057004C
:1068B000F1A159005A005B005C005D005E005F00C2
:1068C00060006100620063006400650036006700DC
:1068D000680069006A006B006C006D006E006F005C
:1068E00070007100720073003100E5008A008B00B7
:1068F000E000E100E200E300F1A1E500E600E700CE
:106900000100010001000100EA4401000100E2442D
:106910000100010001000100460001004A004B0097
:10692000010001004700480001000100E9440100A6
:106930000100010001000100010001003A003B00DC
:106940003C003D003E003F0040004100420043004B
:10695000010035004C0039000100440045005200A0
:1069600001000100010050004F0029004D004E00C1
:106970005100010044004500010001000100010038
:106980000100010044004500010001000100010078
:1069900001000100010001004900010001004D005B
:1069A0004A004E004B000100010001005400550058
:1069B00001000100010001000100010001000100CF
:1069C0000100010001000100010001006700010059
:1069D00001000100010001000100010001000100AF
:1069E0000100010001000100490001000100010057
:1069F000010001000100010001000100010001008F
:00000001FF
